:020000040000FA
:10000000000000308A001A280528F4000308F500D3
:10001000F10B14280A30F10072082F3AF200850023
:1000200073083F3AF30086000B1175088300F40E45
:10003000740E090081018B0185018601831603136B
:1000400085018601D530810006309F00831203139D
:100050008B168B172530F2001530F3000A30F100B3
:10006000302800340034FF3FFF3FFF3FFF3FFF3F9A
:10007000FF3FFF3FFF3FFF3FFF3FFF3FFF3FFF3F90
:10008000FF3FFF3FFF3FFF3FFF3FFF3FFF3FFF3F80
:10009000FF3FFF3FFF3FFF3FFF3FFF3FFF3FFF3F70
:1000A000FF3FFF3FFF3FFF3FFF3FFF3FFF3FFF3F60
:020000040000FA
:1042000012003400FF00FF00FF00FF00FF00FF006E
:10421000FF00FF00FF00FF00FF00FF00FF00FF00A6
:10422000FF00FF00FF00FF00FF00FF00FF00FF0096
:10423000FF00FF00FF00FF00FF00FF00FF00FF0086
:10424000FF00FF00FF00FF00FF00FF00FF00FF0076
:10425000FF00FF00FF00FF00FF00FF00FF00FF0066
:10426000FF00FF00FF00FF00FF00FF00FF00FF0056
:10427000FF00FF00FF00FF00FF00FF005600780076
:020000040000FA
:02400E003B3B3A
:020000040000FA
:084000001200340056007800A4
:00000001FF
